:1000000000308A005F280000FF00030E8301A1007A
:100010007F08A0000A08A8008A01A00E0408A20018
:100020007708A3007808A4007908A5007A08A6003C
:100030007B08A700831383128C308400801D222844
:100040008C193528220884002308F7002408F800BA
:100050002508F9002608FA002708FB0028088A006E
:10006000210E8300FF0E7F0E09008A1143280A101B
:100070008A100A118207023406340E341E343E34CC
:100080007E34FE34FF34290893008C118A11222813
:100090002F308400000803195E280130F800BF30BB
:1000A000F7006400F70B5128F80B4F284A30F7008F
:1000B000F70B582800006400800B4D2800348401A1
:1000C0001F308305603083168F001F129F121B089C
:1000D00080399B0007309C000108C03981000E3038
:1000E000F700073083128101813084000008F03965
:1000F0000738800064000008F739F719F0397704F1
:10010000800083161F129F121B088039D2389B0073
:100110001F1383121F179F1783169F1383121F1419
:10012000941283160611861406120030831294006E
:100130008316940083129001073083169C000508F3
:1001400064000230F700F70BA328000000001C0831
:1001500083120D1383169D01861183128611831657
:100160000611831206118316861083128610203022
:10017000F8001F08C73978049F009501831686117F
:10018000831286110C3097000030F800043892007A
:1001900064308316920062308F0002308312950023
:1001A00083168610831286106430AF0048208316B1
:1001B0008610831286141430AF0048201F151F19B3
:1001C000DF281E08783C031CD02883168610831273
:1001D00086100830F8001F08C73978049F006400B3
:1001E0002030F700F70BF228000000001F151F1940
:1001F000F7281E08F7000310F70C7708283EAC001C
:1002000095010030F800043892002C088316920003
:100210001430831295003230AE00FA30AF0048201F
:10022000AE0B0D2983169401223083129400023004
:10023000A90029089300C0308B0483168C15831203
:10024000AA012A08073C031C2E292A083720F80097
:10025000A9003730AF004820AA0A2129831694014B
:100260008312940183168C110611831206150A302D
:10027000AE008230AF004820AE0B3929831606113C
:080280008312061142296300FC
:04400E003C2FFC3F08
:00000001FF
